:10000000D42864001720031801288920A80108308B
:10001000A3008A2017200318A80AAB1EA801A20C6F
:10002000A30B0928AB1AA2138A202208080036085D
:100030008400340884178004841300052B1B3406C5
:10004000FF3E0800A401A501B312CA20D33E031944
:10005000B3162D3EC63E031825280A3E031C25284C
:10006000A2000310240DA000250DA100200DA10D5C
:10007000A4070318A10A2108A507A40DA50D2208AD
:10008000A4070318A50AA90303194D28CA20C63ED0
:1000900003184D280A3E03183028B31E5428A4091B
:1000A000A509A40A0319A50A2408CF28A600360822
:1000B00084008030B3050830A70003100318B30A8A
:1000C0006F20A60CA70B5E280000AB1A330C6F2024
:1000D000D22003146F202F08A3002E08A128841318
:1000E000AB1F7E28000834042B1F340680008417C1
:1000F00000083404031C340680008A2800083404F5
:10010000031C34062B1B3406800084173409800539
:100110008A2833172B081F39FF3EA1002A08F53E15
:100120000318A10A331FAE283313A0000230C520E4
:10013000AE2883178001840AFF3E031D9A28CF282A
:10014000A301A200FF30A207031CA307031CCF28B2
:100150000330A100DF30AE20A228A101E83EA000BC
:10016000A109FC30031CB728A0070318B428A00776
:100170006400A10FB4282018BD28A01CC1280000CD
:10018000C12808000310A10CA00CFF3E0318C228D0
:100190002008CF28840031088A00300882008313A9
:1001A00003138312640008002030840060308A0149
:1001B0009A20A030840050308A019A2010308400A8
:1001C00060308A0199209030840060308A01992043
:1001D000C8308A01A0200730B6004030B4002D306E
:1001E000AA000330AB00AE01AF016D308A0156208A
:1001F0000730B6008030B4002D30AA000330AB00C9
:100200008A010120523C8A110A12031D0029A9010A
:100210000130B000B1018A012220C1000730B600D0
:100220008030B4002D30AA000330AB008A010120D9
:100230004A3C8A110A12031D16298A010120313C09
:100240008A110A12031D16298A010120463C8A11CF
:100250000A12031D1629A9010130B000B1018A015B
:100260002220BB000730B6008030B4002D30AA0039
:100270000330AB008A0101204A3C8A110A12031D97
:100280003A298A010120323C8A110A12031D3A29B7
:100290008A010120463C8A110A12031D3A29A9014C
:1002A0000130B000B1018A012220BD000730B60044
:1002B0008030B4002D30AA000330AB008A01012049
:1002C0004A3C8A110A12031D5E298A010120333C2F
:1002D0008A110A12031D5E298A010120463C8A11F7
:1002E0000A12031D5E29A9010130B000B1018A0183
:1002F0002220BF000730B6008030B4002D30AA00A5
:100300000330AB008A0101204A3C8A110A12031D06
:1003100082298A010120313C8A110A12031D822997
:100320008A010120523C8A110A12031D8229A90167
:100330000130B000B1018A012220BC000730B600B4
:100340008030B4002D30AA000330AB008A010120B8
:100350004A3C8A110A12031DA6298A010120323C57
:100360008A110A12031DA6298A010120523C8A1112
:100370000A12031DA629A9010130B000B1018A01AA
:100380002220BE000730B6008030B4002D30AA0015
:100390000330AB008A0101204A3C8A110A12031D76
:1003A000CA298A010120333C8A110A12031DCA2975
:1003B0008A010120523C8A110A12031DCA29A9018F
:1003C0000130B000B1018A012220C0008A110A1256
:1003D000E9213B083D07B800B901B90D3F08B8074E
:1003E0000318B90A3C08B8070318B90A3E08B80749
:1003F0000318B90A40083807C20064004208003CEC
:100400008A110A12031D062A8A01EB2864000130B2
:100410003B028A110A12031C602A08158316081170
:100420008312881183168811831207168316071208
:100430008312871283168712831241088A01A02033
:1004400008158316081183128811831688118312E8
:1004500007128316071283128716831687128312D8
:1004600041088A01A02008118316081183128815FB
:1004700083168811831207128316071283128716B8
:1004800083168712831241088A01A020081183165F
:100490000811831288158316881183120716831694
:1004A00007128312871283168712831241088A016A
:1004B000A020BB038A110A1264228A110A12632A3D
:1004C0008A110A1264220800640001303D028A1178
:1004D0000A12031CBE2A06168316061283128612FF
:1004E0008316861283120617831606138312861349
:1004F00083168613831241088A01A02006168316EC
:10050000061283128612831686128312061383162E
:1005100006138312861783168613831241088A01F5
:10052000A0200612831606128312861683168612E0
:1005300083120613831606138312861783168613F7
:10054000831241088A01A020061283160612831224
:1005500086168316861283120617831606138312D5
:10056000861383168613831241088A01A020BD03D7
:100570008A110A12C2228A110A12C12A8A110A1287
:10058000C2220800640001303F028A110A12031CD3
:100590001C2B0614831606108312861083168610F1
:1005A000831206158316061183128611831686118F
:1005B000831241088A01A0200614831606108312B4
:1005C0008610831686108312061183160611831275
:1005D000861583168611831241088A01A020061011
:1005E0008316061083128614831686108312061152
:1005F000831606118312861583168611831241080D
:100600008A01A02006108316061083128614831612
:10061000861083120615831606118312861183161F
:100620008611831241088A01A020BF038A110A1291
:1006300020238A110A121F2B8A110A122023080074
:10064000640001303C028A110A12031C7A2B081143
:1006500083160811831288158316881183120712D6
:100660008316071283128716831687128312410896
:100670008A01A02008158316081183128811831699
:1006800088118312071283160712831287168316A6
:100690008712831241088A01A020081583160811C9
:1006A0008312881183168811831207168316071286
:1006B0008312871283168712831241088A01A020B1
:1006C0000811831608118312881583168811831266
:1006D0000716831607128312871283168712831256
:1006E00041088A01A020BC038A110A127E238A11C4
:1006F0000A127D2B8A110A127E2308006400013041
:100700003E028A110A12031CD82B06128316061207
:100710008312861683168612831206138316061317
:100720008312861783168613831241088A01A0203C
:1007300006168316061283128612831686128312F9
:1007400006138316061383128617831686138312E5
:1007500041088A01A020061683160612831286120B
:1007600083168612831206178316061383128613C6
:1007700083168613831241088A01A020061283166D
:1007800006128312861683168612831206178316A4
:1007900006138312861383168613831241088A0177
:1007A000A020BE038A110A12DC238A110A12DB2B55
:1007B0008A110A12DC2308006400013040028A1109
:1007C0000A12031C352C0610831606108312861499
:1007D000831686108312061183160611831286155E
:1007E00083168611831241088A01A02006148316FD
:1007F0000610831286108316861083120611831644
:1008000006118312861583168611831241088A0108
:10081000A0200614831606108312861083168610F5
:10082000831206158316061183128611831686110C
:10083000831241088A01A020061083160610831235
:1008400086148316861083120615831606118312EA
:10085000861183168611831241088A01A020C003E5
:100860008A01E9218A110A12372C8A01E92108003C
:0608700063008A01382C30
:02400E007D3FF4
:00000001FF
